:100000000C9450050C94B1050C9494080C94B10513
:100010000C94B1050C94B1050C94B1050C94B10588
:100020000C94B1050C94B1050C9412160C94B10506
:100030000C94C1230C94B1050C94B1050C94B1053A
:100040000C94B1050C94B1050C94B1050C94B10558
:100050000C94B1050C9416240C94B1050C94B105C4
:100060000C94B1050C94B1050C94B1050C94B10538
:100070000C94B1050C94B1050C94B1050C94B10528
:100080000C94B1050C94B1050C94B1050C94B10518
:100090000C94B1050C94B1050C94B1050C94B10508
:1000A0000C94B1050C94B1050C94B105660A680A6C
:1000B000740A740A740A740A740A740A6A0A6C0A62
:1000C0006E0A740A740A680A760A740A740A300A94
:1000D000660A740A740A6C0A740A740A740A740A46
:1000E000740A740A6E0A660A520A740A560A740A74
:1000F000740A740A320A6A0A740A740A600A740A70
:10010000740A740A340A720A740A540A740A680A6D
:10011000740A740A640A580A740A5A0A6C0A740A3D
:10012000740A740A620A5C0A740A740A740A740A09
:10013000740A740A740A5E0A740A360A740A740A23
:100140006A0A740A740A720A740A740A740A740ACB
:10015000740A740A740A740A740A380A740A740AEB
:10016000740A600A740A740A740A740A740A740AB3
:10017000740A740A740A740A3A0A740A3C0A3E0A37
:10018000740A740A740A400A420A440A740A460A43
:10019000480A740A740A740A700A4A0A740A4E0AEF
:1001A0004C0A500A740A740A740A740A720A9A0A87
:1001B000A80AB40AB40A8C0AB40AB40AB40AB40A83
:1001C000B40AB40AB40AB40AB40AB40AB40AB40A3F
:1001D000B40A8E0AB40A900AB40AB40AB40AB40A79
:1001E000AC0AB40AC30AAA0AB40AB40AB40AB40A22
:1001F000B40AB40AB40AB40AB40AB40AB40AB40A0F
:10020000B40A840AA00A920AA40AB40A940AB40A94
:10021000980AB40AA20A960AA60A9C0A9E0AB40A76
:10022000B40AB40AB40AB40AB40AB40A860A880A38
:100230008A0AAE0AB00AB40AB40AB40AB20A920B25
:10024000B00BBC0BE00BF00BFC0B180C2F0C520C82
:100250006F0CFA0C260DA00DD20DBC0DE30DF50DA3
:10026000FD0D030E070E0D0E690E6B0E6D0E6F0E5B
:10027000AF0E770E770E770E710E730E750E60143B
:1002800087147F1587147F15D314F6147F154D1529
:100290005C15D819D819021A021A5D1A881C881C14
:1002A000881C911A881C7C1B7C1B421C881C571CB8
:1002B000751C007B46010203763A687F6577482B00
:1002C000353B6978796439141E3C6A7A1D16041A24
:1002D0001F3D6B061B070821203E6C2C19091715C2
:1002E000223F6D11050B0A1C23406E7E100D182451
:1002F00025416F360E0C122726427037380F331304
:100300002D43717534322F2E44727C7D2830317428
:10031000457351504A524D492A5466594F5C5F4CBF
:100320004B4E62635A5D5E60295367585B56576156
:1003300047554842403E3C3A3B456843413F3D2B90
:10034000357E697A790078141E7C6A7B1D16041A42
:100350001F7F6B061B070821204D6C2C19091715F0
:10036000224A6D11050B0A1C234C6E49100D1824EE
:1003700025516F360E0C1227264F7037380F331366
:100380002D52717534502F2E4E72397D28306531C3
:100390004B735464586776012A773259745C5F66F0
:1003A000020362635A5D5E60295344575B56556190
:1003B000474680291E1F20212223242526272D2E53
:1003C0002A2B141A0815171C180C12132F30287812
:1003D000041607090A0B0D0E0F33343579311D1B36
:1003E00006190511103637387D557A2C393A3B3CC1
:1003F0003D3E3F4041424353475F6061565C5D5E16
:1004000057595A5B62634648324445677B7F6503B0
:1004100001025250514F68696A6B6C6D6E6F70715A
:10042000725800494C754A4D734B4E767C777E74FA
:10043000665472253032582000623A2530345820F4
:1004400000652530325820002146554C4C212000B3
:100450002146462120007725303258200021435381
:10046000335F4630210A00214353335F52454144F4
:1004700059210A00214353325F45305F4630210A3B
:1004800000214353325F4630210A00214353325F3B
:100490004530210A00214353325F494E4954210A15
:1004A00000214353315F45305F25303258210A0027
:1004B0000A5B4F56525D20004C2575200053257570
:1004C00020000A49443A2530345828256429200060
:1004D0004D6F7573653A206E6F7420737570706F11
:1004E000727465640A005225752000572575200036
:1004F0005725752000572575200058257520004187
:100500002575200049257520005B4348475D200084
:100510000A5052543A25303258204953523A253025
:10052000345820005B5253545D20000A4552523A21
:1005300025303258204953523A2530345820000A89
:100540004B6579626F6172642073746172742E0AF4
:10055000000A55534220636F6E6669677572656461
:100560002E0A000A0A544D4B3A30616230656266C9
:10057000382F4C5546410A0A003403490042004DC9
:100580000020005000430020006B006500790062ED
:10059000006F00610072006400200063006F006E55
:1005A0000076006500720074006500720000000EA5
:1005B0000374002E006D002E006B002E000000045E
:1005C00003090409027400040100A03209040000B8
:1005D000010301010009211101000122400007056A
:1005E000810308000A090401000103000000092139
:1005F000110100012236000705820308000A0904E0
:100600000200020300000009211101000122220062
:1006100007058303200001070503032000010904E7
:10062000030001030000000921110100012239002B
:10063000070584032000011201100100000008EDED
:10064000FEEE1B01000102000105010906A10105E2
:100650000719E029E71500250195087501810205B4
:1006600008190129059505750191029501750391F8
:10067000010507190029F71500250195F875018175
:1006800002C00631FF0974A1010975150026FF009B
:100690009520750881020976150026FF00952075C2
:1006A000089102C005010980A101850216010026FA
:1006B00037001A81002AB700751095018100C00526
:1006C0000C0901A1018503160100269C021A0100F4
:1006D0002A9C02751095018100C005010906A1013F
:1006E000050719E029E71500250195087501810224
:1006F0009501750881010508190129059505750100
:1007000091029501750391010507190029FF150054
:1007100026FF00950675088100C0636F6E73756DC6
:1007200065723A20253034580A0073797374656D08
:100730003A20253034580A000A002530325820006B
:100740006B6579626F6172643A20004C45443A20CF
:10075000253032580A00253032583A202530386288
:1007600025730A00722F6320303132333435363727
:100770000A0064656C5F6B65795F6269743A206337
:10078000616E27742064656C3A20253032580A0067
:100790006164645F6B65795F6269743A2063616E5E
:1007A0002774206164643A20253032580A003F00E3
:1007B000433E20004C25640A000A092D20436F6E39
:1007C000736F6C65202D0A4553432F713A0971757B
:1007D00069740A000A092D204D61676963202D0A9A
:1007E000643A0964656275670A783A0964656275F6
:1007F00067206D61747269780A6B3A096465627585
:1008000067206B6579626F6172640A6D3A0964658D
:10081000627567206D6F7573650A763A0976657241
:1008200073696F6E0A733A097374617475730A633E
:100830003A09636F6E736F6C65206D6F64650A3083
:100840002D343A096C61796572302D342846313087
:100850002D4634290A506175733A09626F6F746CC2
:100860006F616465720A6E3A094E4B524F0A003F3F
:10087000004E4B524F3A206F66660A004E4B524F65
:100880003A206F6E0A0074696D65725F726561640B
:10089000333228293A202530346C580A006B6579A8
:1008A000626F6172645F6E6B726F3A2025580A0046
:1008B0006B6579626F6172645F69646C653A20256B
:1008C000580A006B6579626F6172645F70726F7451
:1008D0006F636F6C3A2025580A00686F73745F6B02
:1008E0006579626F6172645F6C65647328293A2070
:1008F00025580A000A092D20537461747573202D40
:100900000A004743433A20352E342E3020415652B8
:100910002D4C4942433A20322E302E30204156523F
:100920005F415243483A20617672350A004F505475
:10093000494F4E533A204C55464120455854524158
:100940004B455920434F4E534F4C4520434F4D4D3F
:10095000414E44204E4B524F204B45594D41505F24
:1009600053454354494F4E20424F4F544C4F4144FE
:1009700045525F53495A450A004255494C443A2072
:100980003061623065626638202831313A35373A55
:100990003138204D61792032322032303230290A0C
:1009A000005649443A2030784645454428742E6D17
:1009B0002E6B2E29205049443A20307831626565EB
:1009C0002849424D205043206B6579626F61726403
:1009D00020636F6E76657274657229205645523AAF
:1009E000203078303030310A00444553433A206398
:1009F0006F6E766572742049424D205043206B65BE
:100A000079626F61726420746F205553420A000A44
:100A1000092D2056657273696F6E202D0A000A6DCC
:100A20006F7573653A206F66660A000A6D6F75739D
:100A3000653A206F6E0A000A6B6579626F617264B5
:100A40003A206F66660A000A6B6579626F617264AC
:100A50003A206F6E0A000A6D61747269783A206FED
:100A600066660A000A6D61747269783A206F6E0AD0
:100A7000000A64656275673A206F6E0A000A646551
:100A80006275673A206F66660A000A0A626F6F74C1
:100A90006C6F616465722E2E2E2000433E20000094
:100AA00011241FBECFEFDAE0DEBFCDBF04B603FED8
:100AB00041C08091880390918903A0918A03B091ED
:100AC0008B038730904BA740B04BA1F51092880361
:100AD0001092890310928A0310928B0314BE0FB6F2
:100AE000F894A895809160008861809360001092CE
:100AF00060000FBE1092010810920008E3E0F0E0E1
:100B000089E080935700E491E695E370E150E3308B
:100B100040F4F0E0EE0FFF1FE35DFE4F8081918116
:100B200002C080E090E1E0E0F0E8E81BF90BF69508
:100B3000E795099511E0A0E0B1E0E6E3FCE402C02E
:100B400005900D92A433B107D9F723E0A4E3B1E0F7
:100B500001C01D92A838B207E1F70E9475110C94EC
:100B600019260C940000FF93EF93E0913401F0916B
:100B70003501309709F00995EF91FF910895FC0137
:100B80008591803011F0EFDFFBCF0895FF27E0E281
:100B900030E247FF0CC0419597FF09C0EDE2609538
:100BA000709580959095611D711D811D911D27FF88
:100BB00002C0219530E350E2AA27660F771F881FF5
:100BC000991FAA1FA41710F0A41B63955A95A9F7A3
:100BD000AA3008F0A95FA05DAF93F3956115710588
:100BE0008105910541F7ED3211F4EF93F395F2177A
:100BF00018F43F93F395FBCF8F91B5DFFA95E1F7AA
:100C00000895E991F9918591803021F0853219F0AC
:100C1000AADFF9CF089520E0E89455915532C1F349
:100C2000503311F4689455915A3348F4505390F36B
:100C3000220F022E220F220F200D250FF4CF0EF4CB
:100C4000219589919991533619F3533729F15335E9
:100C500059F1BC0188279927E8945C3621F48991E1
:100C6000999168945591543639F446EF7EF077FFA8
:100C70000DC08FEF9FEF0AC055374AE039F0583565
:100C800040E121F0523642E009F00895FF93EF93DE
:100C90007DDFEF91FF91B7CFFF93EF93FC0181913F
:100CA0008030B9F360DFFBCFFF93EF9368DFF1CFC4
:100CB000DF93CF93CDB7DEB72596A3DFCF91DF913A
:100CC0000895282F80914101823071F08330B1F076
:100CD000813001F5E62FF0E038E0739FE00DF11D63
:100CE0001124EE54FC4F13C0E62FF0E088E0789F0B
:100CF000E00DF11D1124EE5CFC4F09C0E62FF0E081
:100D000038E0739FE00DF11D1124EE54FD4FE49186
:100D1000E03819F480E090E008959E2F9077892FB5
:100D200090E034E0959587953A95E1F738E0239F78
:100D3000800D911D112444E0880F991F4A95E1F719
:100D4000EF709C012E0F311DF901EE0FFF1FE050D7
:100D5000F8498591949108955998519A0895519818
:100D6000599A08955898509A08955098589A089505
:100D70005198599A85E08A95F1F7000089B18695D6
:100D8000817008955098589A85E08A95F1F700008F
:100D900089B181700895CF93DF93EC010E94B8066A
:100DA000882341F0209731F085E08A95F1F7000023
:100DB0002197F4CFCE01DF91CF910895CF93DF93A8
:100DC000C2E3D0E00E94B806811108C0209731F03C
:100DD00085E08A95F1F700002197F4CFCE01DF91ED
:100DE000CF9108952E9826982F9827980E94AC06A8
:100DF0000E94B506E9E6F0E0808188608083E9988A
:100E00000895E19AE99A0E94AF060C94B506E99814
:100E10000E94AC060C94B506CF93DF932FB7F894DD
:100E2000C0910201D0910301CE01882781159F4F07
:100E300019F080E09FEF02C08FEF90E08C2B9D2B8C
:100E400090930301809302012FBFCE0199278F3F1A
:100E5000910581F5CD2FDD27C03FD10551F0CF3F62
:100E6000D10509F451C080917503C034D10599F4BE
:100E700007C08091750380FF33C080E594E004C013
:100E800080FF2EC088E494E09F938F930E945806C1
:100E90000F900F9025C080FF37C0DF93CF9381E480
:100EA00094E09F938F930E9458060F900F900F909D
:100EB0000F902AC0CE018F6F019699F08091750333
:100EC00080FF0CC0DF93CF9389E394E09F938F93CF
:100ED0000E9458060F900F900F900F90CD2F01C0D9
:100EE000CFEF8091750380FF0CC01F92CF9382E3F8
:100EF00094E09F938F930E9458060F900F900F904D
:100F00000F908C2F90E002C08FEF9FEFDF91CF9179
:100F10000895CF93CAE1C15069F00E940C078F3F3A
:100F20002FEF920749F48FE99FE00197F1F700C096
:100F30000000F1CF8FEF9FEFCF91089510923A010B
:100F400010923901109238011092370180E090E838
:100F500090930101809300018FEF9FEF9093030125
:100F6000809302010895EF92FF920F931F93CF9306
:100F7000DF93082F109237018091750380FF0CC01A
:100F80001F920F9386E594E09F938F930E945806DB
:100F90000F900F900F900F90E9980E94AC060E945E
:100FA000B5068FE891E00197F1F700C000000E94BC
:100FB000B2068FE891E00197F1F700C000000E94AF
:100FC000AF0680E197E20E94CB06892B11F481E005
:100FD0007FC0C0E0D0E0FF24F39410E0EE24E3945F
:100FE00090E59A95F1F7C8010C2E02C0959587956A
:100FF0000A94E2F780FF04C0FE240E94B50602C0F6
:101000000E94B2060E94DE06892B11F482E060C0C5
:1010100082E390E00E94CB06892B11F483E058C054
:101020002196C830D105E1F680E58A95F1F7FF20D9
:1010300019F00E94B50602C00E94B2060E94DE06A8
:10104000892B11F484E044C082E390E00E94CB0637
:10105000892B11F485E03CC090E59A95F1F70E9448
:10106000B5060E94DE06892B11F486E031C082E3CA
:1010700090E00E94CB06892B19F0C2E3D0E009C0B2
:1010800087E026C0209759F025E02A95F1F7000067
:1010900021970E94C2068111F5CFCD2B11F488E073
:1010A00017C00E94DE06892B19F0C2E3D0E009C008
:1010B00089E00EC0209759F085E08A95F1F700008D
:1010C00021970E94C2068823A9F3CD2BB9F48AE0A8
:1010D00080933701809137018061809337010E94AE
:1010E000AF060E94B506E19AE99A8FEF9FEFDF9174
:1010F000CF911F910F91FF90EF9008958FEF9FEF89
:1011000090930301809302010E949E070E94AF0604
:101110000E94B506E19AE99ADF91CF911F910F9154
:10112000FF90EF900C9489071F920F920FB60F92C9
:1011300011242F933F934F935F938F939F9329B1E4
:101140009091760340910001509101014115504862
:1011500019F49093360111C080913601981769F007
:101160008F5F981751F08091000190910101909349
:101170003A018093390180E2DDC0809100019091B5
:10118000010196958795909301018093000120FFBE
:1011900009C0809100019091010190689093010134
:1011A000809300018091000190910101992780387E
:1011B000910509F4F9C0A8F48032910509F4F4C04E
:1011C00038F4009709F4F0C0409709F489C0A9C029
:1011D0008034910509F4E8C08035910509F480C098
:1011E000A0C0803C910539F150F48039910509F493
:1011F00077C0803A910509F094C084E64DC0803DE7
:10120000910509F46DC0803E910509F08AC0809176
:1012100000019091010190933A01809339018091EE
:10122000000190910101892F9927909301018093EA
:10123000000183E252C084E649990FC0882369F017
:1012400095E09A95F1F700008150F6CF882349F098
:1012500095E09A95F1F7000081504999F7CF8111F7
:10126000A3C0809100019091010190933A01809375
:1012700039018091000190910101892F9927909364
:1012800001018093000182E228C0882379F095E073
:101290009A95F1F700008150499BF7CF07C088234A
:1012A00049F095E09A95F1F7000081504999F7CF00
:1012B00081117AC0809100019091010190933A01CF
:1012C000809339018091000190910101892F992724
:1012D000909301018093000181E28093380133C033
:1012E000809100019091010190933A01809339011E
:1012F000809100019091010197FF02C080E101C03F
:1013000081E180933801809100019091010146E0D4
:10131000969587954A95E1F7909301018093000196
:1013200012C0809100019091010190933A01809345
:10133000390180E8809337018091370190E0982F40
:1013400088278F6F27C08091000190910101992714
:101350008F3F910511F480EFEDCF809103018F3F16
:1013600031F0809102018F3F11F080E4E3CF809152
:10137000020190910301982F882790930301809395
:1013800002012091000130910101809102019091B0
:101390000301822B909303018093020180E090E887
:1013A00090930101809300019F918F915F914F91E4
:1013B0003F912F910F900FBE0F901F901895CF93D4
:1013C000C82F8DEE0E94B3078A3F910521F48C2F20
:1013D000CF910C94B307CF910895E82FE695E69549
:1013E000E695EF70F0E0EB5BFE4F4081282F277011
:1013F00081E090E002C0880F991F2A95E2F7242F20
:1014000030E028233923232B11F4842B8083089583
:10141000E82FE695E695E695EF70F0E0EB5BFE4F82
:101420002081382F377081E090E002C0880F991F2B
:101430003A95E2F7422F50E048235923452B19F003
:101440008095822380830895482F50E0FA013397D6
:10145000E138F10508F048C0EA5AFF4F0C94132612
:1014600087E108958FE108958CE5089580E6089559
:1014700082E6089587E2089583E508958FE208954E
:1014800089E3089587E308958FE3089587E4089535
:101490008FE4089586E508958EE508958FE7089511
:1014A00080E0089585E608958EE608958FE6089514
:1014B00080E3089588E3089580E4089588E408951A
:1014C00080E5089587E508958FE5089588E10895FA
:1014D00088E0089580E2089580E1089589E1089503
:1014E0008DE6089588E208958F7708958FE0089536
:1014F000CF93482F50E0FA017C97E834F105A0F52E
:10150000E952FF4F0C94132685E53EC08AE53CC0A6
:101510008BE53AC08CE538C08DE536C08EE534C029
:101520008FE532C080E630C081E62EC082E62CC056
:1015300083E62AC08FE628C081E726C082E724C060
:1015400084E722C085E720C087E71EC088E71CC06B
:101550008AE71AC08CE718C08FE716C080E714C06E
:1015600089E712C08BE710C0C82F1F928F9381EAC2
:1015700094E09F938F930E9458060F900F900F90C6
:101580000F908C2F01C084E5CF9108950F931F9386
:10159000CF93DF930E94EF238C010E940C07EC0194
:1015A000019631F4C8010E940724843F9140A8F3BA
:1015B000CE01DF91CF911F910F9108950E94F20605
:1015C0000C94010780917503816080937503E5E4B5
:1015D000F1E0119281E0E535F807D9F70895E82F99
:1015E000F0E0EB5BFE4F80810895E5E4F1E01192BD
:1015F00081E0E535F807D9F70895982F80914101EA
:10160000823048F092FB882780F990FD826091FD3E
:1016100084600C94DF090895CF93DF9380913701A4
:10162000882371F18091390190913A01209137011D
:101630009F938F931F922F938BE295E09F938F93AD
:101640000E9458068091370180750F900F900F907F
:101650000F900F900F9071F4809140018B3051F4F6
:1016600084E295E09F938F930E9458061092400168
:101670000F900F901092370110923A011092390199
:1016800080913801882309F440C0909138018091FD
:1016900044019817D1F18091390190913A0120913C
:1016A00038019F938F931F922F9380E195E09F9332
:1016B0008F930E945806809144010F900F900F90D5
:1016C0000F900F900F9085FF04C09091380194FD0A
:1016D00006C084FF12C08091380185FF0EC0809142
:1016E00040018B3051F489E095E09F938F930E94E5
:1016F0005806109240010F900F908091380180930E
:10170000440110923A0110923901E09140018E2F6C
:1017100090E08C30910508F026C3FC01E15EFE4F9D
:101720000C9413260E9407070E94EF239F938F9328
:1017300084E095E09F938F930E9458061092410198
:1017400010924301109242010E94F50A0E948819EA
:101750000E94EF2390933F0180933E0181E065C09A
:1017600080913E0190913F010E940724893E934061
:1017700008F4F9C282E031C00E949E070E9401076E
:101780008FE99FE00197F1F700C000008FEF0E9402
:10179000B3078A3F910511F486E001C083E080938E
:1017A00040010E94EF239F938F938FEF94E09F93CC
:1017B0008F930E9458060F900F900F900F90D3C2F6
:1017C0000E9407072E98269A2F98279A0E94EF23A7
:1017D00090933F0180933E0184E080934001C3C217
:1017E00080913E0190913F010E940724853F9140E6
:1017F00008F4B9C285E0F1CF2E9826982F98279843
:101800000E949E070E9401070E94EF239F938F93DF
:101810008AEF94E09F938F930E9458060E94EF23D3
:1018200090933F0180933E0186E080934001C3CFB7
:101830000E940C07019609F496C20E94EF239F9321
:101840008F9385EF94E09F938F930E9458060E9498
:10185000EF2390933F0180933E0187E0E6CF809194
:101860003E0190913F010E940724853F914018F06E
:1018700089E0809340010E940C07019609F473C22D
:101880000E94EF239F938F9380EF94E09F938F9319
:101890000E9458060E94EF2390933F0180933E01DF
:1018A00088E0C3CF80913E0190913F010E940724C0
:1018B000853F914018F089E0809340010E940C0719
:1018C000019609F450C20E94EF239F938F938BEEF1
:1018D00094E09F938F930E94580689E0A6CF82EFF1
:1018E0000E94B3078F3F2FEF920789F08A3F91053F
:1018F00089F40E94C60A8F3F3FEF930771F0D82FFB
:10190000CC270E94C60A9E01282BC90108C08FEF70
:101910009FEF05C08EEF9FEF02C080E090E09093B4
:101920004301809342010E94EF239F938F9386EEA1
:1019300094E09F938F930E9458068091420190916A
:1019400043010F900F900F900F90009711F482E0D9
:101950002BC08F3F3FEF930711F481E025C08E3FEE
:101960002FEF9207A1F38F3F910559F480ED94E09A
:101970009F938F930E945806109241010F900F90F1
:101980001FC09C0125583B4A2230310580F480EF6E
:101990000E94B3078A3F9105D1F683E00E94B30706
:1019A0008A3F9105A1F683E08093410109C0803B05
:1019B0003FEB9307C1F3882781159F4BA1F3C7CF56
:1019C000809141011F928F93809143018F93809169
:1019D00042018F9382EC94E09F938F930E9458066C
:1019E0008AE0809340010F900F900F900F900F901E
:1019F0000F90B9C10E94EF239F938F938DEB94E0DA
:101A00009F938F930E9458060F900F900F900F9006
:101A100080914101823029F0833039F488EF0E94AF
:101A2000B3070E9400170E94FD0A8BE080934001DB
:101A30000E94EF239F938F9388EB94E09F938F9363
:101A40000E9458060F900F900F900F900E940C0765
:101A50009C012F3F9FEF390709F485C121153105FE
:101A600019F02F3F310569F40E94F50A0E94881988
:101A700080EB94E09F938F930E9458060F900F90F5
:101A800072C190914101923009F44DC0933009F434
:101A9000CCC0913009F067C190913D01923099F02E
:101AA00028F4992341F09130C1F03AC0933081F18C
:101AB000943091F135C0803E21F0813E51F482E0B6
:101AC00005C081E003C08D31F9F483E080933D01CE
:101AD0004AC187FFE4C08F770EC1863309F118F43D
:101AE0008A3229F41DC08A3AD9F0863BC9F087FDB5
:101AF00005C00E94780A0E94ED0912C08F770E94EB
:101B0000780A0E94080A0CC08D3951F484E0DECFB7
:101B1000853431F485E5C3C0853411F485E5EBC027
:101B200010923D0120C1E0913C014E2F50E0493020
:101B3000510508F077C0FA01E55DFE4F0C941326BD
:101B4000803E69F030F4833871F0843871F48FE7A7
:101B500057C0813E31F0803F41F481E05BC082E0BC
:101B600059C084E057C082E04BC087FF98C00E94F4
:101B7000F50A85E994E098C0893509F453C0803F9F
:101B800019F0823119F44EC083E044C010923C0138
:101B900087FD03C00E94240A82C00E94F50A8BE8D8
:101BA00094E082C0833821F0843821F48FE738C074
:101BB00082E036C010923C0187FF9DC00E94F50A6A
:101BC00081E894E071C010923C01823109F4CBC0ED
:101BD000893509F4C8C087FD03C00E94240A8BC060
:101BE0000E94F50A84E794E05FC0843121F0803FD1
:101BF000C9F486E00FC085E00DC0873799F480E016
:101C00000E94ED090FC0843169F487E003C0803F72
:101C100049F488E080933C01A6C0873719F480E03E
:101C20000E94080A10923C019EC090913B019130A5
:101C300009F443C038F0923009F463C0933009F4DA
:101C40007FC091C0863809F168F48338D1F020F460
:101C5000803819F582E06CC08438A9F08538E9F441
:101C60008BE01DC08C38A9F030F4873881F08B38B8
:101C7000A1F481E014C08D3871F0803F71F481E0EF
:101C800057C082E00CC08FE70AC086E008C080E041
:101C900006C089E004C08AE002C087FD03C00E943C
:101CA000ED0961C087E694E09F938F930E945806E8
:101CB0000F900F901092400156C0482F50E0FA014B
:101CC000E358F109EB30F10590F4EC5CFE4F0C9415
:101CD000132682E045C08FE743C08BE041C086E019
:101CE0003FC081E03DC089E03BC08AE039C010922E
:101CF0003B0187FD03C00E94080A35C08DE594E0D2
:101D0000D3CF853279F030F4863171F08E3199F489
:101D100080E00BC0863221F0803F69F483E008C088
:101D20008DE503C083E501C081E50E94ED0905C092
:101D300080933B0118C00E94F50A10923B0113C02A
:101D40008E3169F020F48631B1F781E509C0853222
:101D500021F0863281F78DE503C083E501C080E084
:101D60000E94080AEACF81E0DF91CF910895809127
:101D7000790208950895CF93DF9300D01F92CDB7D5
:101D8000DEB720917F03243021F523E029839B8354
:101D90008A8382E08093E9008FEF9091E800815080
:101DA00095FD06C095ED9A95F1F700008111F5CFEC
:101DB0008091E80085FF0DC040E050E063E070E0F6
:101DC000CE0101960E942B138091E8008E778093BC
:101DD000E8000F900F900F90DF91CF910895CF936F
:101DE000DF9300D01F92CDB7DEB720917F03243060
:101DF00029F522E02983805891099B838A832093C7
:101E0000E9008FEF9091E800815095FD06C095EDB7
:101E10009A95F1F700008111F5CF8091E80085FFD8
:101E20000DC040E050E063E070E0CE0101960E94FA
:101E30002B138091E8008E778093E8000F900F902D
:101E40000F90DF91CF910895CF93DF93EC019091A4
:101E50007F03943009F048C0809114018823D9F0A1
:101E6000809115018823B9F09093E90081E88150B1
:101E700049F09091E80095FD05C09AE29A95F1F736
:101E800000C0F5CF8091E80085FF2EC040E050E013
:101E900060E270E019C081E08093E90081E8815040
:101EA00059F09091E80095FD07C0EFE3F1E031971C
:101EB000F1F700C00000F3CF8091E80085FF14C067
:101EC00040E050E068E070E0CE010E942B1380916A
:101ED000E8008E778093E80080E2FE01A9E5B2E099
:101EE00001900D928A95E1F7DF91CF910895CF93FC
:101EF000C0915701C1110BC00E94FB23643C794083
:101F00008105910520F081E080935701C1E08C2F7D
:101F1000CF910895FF920F931F93CF93DF93D82F04
:101F20000FB607FE83C080917F03843081F08091DB
:101F3000070190E001962091090130E0822393236C
:101F40002091080130E08217930709F0CDC00E946C
:101F5000770F811110C08091070190E001962091C8
:101F6000090130E0822393232091080130E0821799
:101F7000930709F0B9C00E94EF238C01C091E900DA
:101F8000CF709091EC00892F817090FD80E8C82B74
:101F900083E08093E90085E0F82E8091EB0085FDD9
:101FA00042C08091EB0080FF3EC08091EE0087FF31
:101FB0003AC08091080190910701981709F457C021
:101FC0009091E80095FF8EC0E0910501F091060127
:101FD000E80FF11D20818F5F909109018923809383
:101FE00008012093F1008091E80085FDE2CF809107
:101FF000E80080FFDECF8091E8008E778093E800D4
:10200000F0920401D6CF8091070190E001962091D3
:10201000090130E0822393232091080130E08217E8
:10202000930709F44CC0CF70C093E90040910701B9
:10203000842F90E001962091090130E082239323C0
:102040002091080130E08217930709F450C0E09115
:102050000501F0910601E40FF11DD0838091070185
:102060008F5F9091090189238093070140C080917F
:10207000E80085FF37C0D093F10021E03091F300F4
:102080008091F20090E0932B892B91F08091E800F1
:1020900080FF0EC08091E80085FF03C01092F10020
:1020A000F9CF8091E8008E778093E800F0920401E8
:1020B000222309F4A8CFCF70C093E90018C0809103
:1020C0000401882309F4AFCF0E94EF239C018017FD
:1020D000910711F4890161CF90910401915090937F
:1020E0000401F8CF20E0CACF40910701B0CF80E0D3
:1020F000DF91CF911F910F91FF90089580917E0302
:10210000811104C00E9497150C94F4150895109243
:102110007E030895089542E061EC81E00E94A412DC
:1021200042E061EC82E00E94A41242E261EC83E0B2
:102130000E94A41242E261EC84E00C94A41280910B
:102140008103833009F455C030F4813071F082305E
:1021500009F48EC008958A3009F47AC08B3009F4EE
:1021600060C0893009F09CC020C080918003813A12
:1021700009F096C08091E800877F8093E800809105
:10218000840390918503892B21F460E289E592E034
:1021900003C060E080E090E070E00E9478138091DE
:1021A000E8008B778093E800089580918003813266
:1021B00009F076C08091840390918503009719F00F
:1021C000039709F06DC08091E800877F8093E80055
:1021D0008091E80082FD05C080917F038111F8CFD6
:1021E0005FC08091F100809379028091E8008B7745
:1021F00053C080918003813A09F052C080918403DA
:1022000090918503892B09F04BC08091E800877F6E
:102210008093E8008091E80080FFFCCF809114015A
:1022200036C0809180038132D9F5809184039091EA
:102230008503892BA9F58091E800877F8093E800CA
:102240000E94D91280918203809314010C94881902
:1022500080918003813221F58091E800877F80930F
:10226000E8000E94D9128091830380937A02089536
:1022700080918003813AA1F48091E800877F809368
:10228000E8008091E80080FFFCCF80917A02809383
:10229000F1008091E8008E778093E8000C94D912C9
:1022A00008958091790280935801109279020E94DA
:1022B000F50A0C9488190C9451110E949C2380916A
:1022C0007D03882329F00E94A92381110C948E128A
:1022D00008950E94BD23809158018093790208954A
:1022E0000C94691108950C947211CF9384B7877F71
:1022F00084BF0FB6F894A8958091600088618093A0
:102300006000109260000FBE90E080E80FB6F89475
:1023100080936100909361000FBE8AE89FE00E9465
:102320006F238AE091E00E94FB1683E695E00E940D
:10233000BF050E94DE0A0E94AF170E9497150E94F7
:10234000F41578940E94B11780917F03843029F0AE
:102350000E94E0160E947211F7CF81E595E00E947D
:10236000BF050E9473118FE395E00E94BF05C3E093
:1023700080917F03853019F40E945D11F9CF0E948E
:10238000B5172091E4003091E500809155019091BE
:1023900056012817390709F468C08091E40090912C
:1023A000E50090935601809355010E94770F882392
:1023B00009F45BC080917F03843009F056C080919E
:1023C000E9008F702091EC00922F917020FD90E831
:1023D000892BC093E9009091EB0090FF43C090914E
:1023E000EE0097FF3FC09091080120910701291747
:1023F00009F12091E80025FF1DC0E0910501F09151
:102400000601E90FF11D30819F5F209109019223A0
:10241000909308013093F1009091E80095FDE3CF8F
:102420009091E80090FFDFCF9091E8009E77909325
:10243000E800D9CF9091F3002091F20030E0392BE1
:10244000232B81F09091E80090FF0CC09091E80060
:1024500095FF03C01092F100F9CF9091E8009E77AC
:102460009093E8008F708093E9000E94E01680CF7F
:10247000292F332723303105C9F060F4213031058D
:1024800081F02230310509F041C084E790E023EC6F
:1024900035E040C021323105E1F02232310531F121
:1024A00035C082E190E027E336E034C099278130DF
:1024B000910549F028F0029749F5E9E7F5E005C0F4
:1024C000EFEBF5E002C0EFEAF5E0849190E09F01C8
:1024D00021C064307105D0F4660F771FFB01EC5DFD
:1024E000FE4F2081318189E090E014C06430710595
:1024F00068F4FB01EE0FFF1FE45EFE4F2081318187
:10250000FB01E85EFE4F808190E004C080E090E037
:1025100020E030E0FA0131832083089580E189BD15
:1025200082E189BD09B400FEFDCF8091D8008F7D86
:102530008093D8008091E00082608093E0008091D9
:10254000E00081FDFCCF0895982F973068F59093B7
:10255000E900981739F07091EC002091ED0050914E
:10256000F00003C0242F762F50E021FD02C09F5FB2
:10257000ECCF3091EB003E7F3093EB003091ED00DB
:102580003D7F3093ED003091EB0031603093EB00F4
:102590007093EC002093ED005093F0002091EE003A
:1025A00027FDE5CF80E008958F708093E90081E0FA
:1025B00008958091800387FF11C08091E80082FD1B
:1025C00005C080917F038111F8CF11C08091E80090
:1025D0008B770BC080917F03882349F08091E800BE
:1025E00080FFF8CF8091E8008E778093E80008950F
:1025F0002091E4003091E50095E64091EC00842FB5
:10260000817040FF23C08091E80080FD1DC0809153
:102610007F03882399F0853099F08091EB0085FD48
:1026200011C04091E4005091E5002417350729F3CB
:10263000915011F09A01E1CF84E0089582E008956D
:1026400083E0089581E0089580E008954091E800D6
:1026500042FFDDCF0895CF92DF92EF92FF920F936A
:102660001F93CF93DF93EC018B017A010E94F81244
:10267000811135C0E114F10439F0F70180819181B5
:10268000081B190BC80FD91FC12CD12C011511051E
:1026900029F18091E80085FD18C08091E8008E77CF
:1026A0008093E8000E94E016E114F10449F0F7017C
:1026B00080819181C80ED91ED182C08285E00FC071
:1026C0000E94F812882311F30AC089918093F100C7
:1026D00001501109FFEFCF1ADF0AD8CF80E0DF9158
:1026E000CF911F910F91FF90EF90DF90CF900895C1
:1026F00020918603309187032617370748F061152C
:10270000710539F42091E8002E772093E80001C08C
:10271000B901FC0120E06115710579F180917F0319
:102720008823F1F18530F1F18091E80083FD3CC010
:102730008091E80082FD2EC08091E80080FFEBCF01
:102740002091F3008091F20090E0922B61157105C9
:1027500051F08830910538F421912093F1006150B7
:1027600071090196F3CF21E0089709F020E08091EC
:10277000E8008E778093E800CECF2111CFCF0AC03A
:1027800080917F03882361F0853061F08091E800BB
:1027900083FD0AC08091E80082FFF2CF80E00895B7
:1027A00082E0089583E0089581E0089520918603F2
:1027B000309187032617370748F06115710539F402
:1027C0002091E8002E772093E80001C0B901FC01B8
:1027D00020E06115710591F180917F03882309F450
:1027E00040C0853009F43FC08091E80083FD3DC0C2
:1027F0008091E80082FD2FC08091E80080FFE9CF42
:102800002091F3008091F20090E0922B6115710508
:1028100059F08830910540F424912093F1003196CD
:10282000615071090196F2CF21E0089709F020E08C
:102830008091E8008E778093E800CBCF2111CCCF38
:102840000AC080917F03882361F0853061F0809118
:10285000E80083FD0AC08091E80082FFF2CF80E0AB
:10286000089582E0089583E0089581E008951F931C
:10287000CF93DF93CDB7DEB7AA970FB6F894DEBF3C
:102880000FBECDBFE0E8F3E08091F100819323E03B
:10289000E838F207C9F70E949F108091E80083FF93
:1028A0002EC18091800390918103492F50E04A30DE
:1028B000510508F024C1FA01E15CFE4F0C94132687
:1028C000803821F0823809F01AC108C080917C0359
:1028D00090917D03992389F082600FC080918403D9
:1028E0008F70873008F00BC18093E9008091EB0076
:1028F00085FB882780F91092E9009091E800977F86
:102900009093E8008093F1001092F100D1C0282F3D
:102910002D7F09F0F4C0882319F0823061F0EFC0F8
:1029200080918203813009F0EAC0933009F080E0A1
:1029300080937D032EC08091820381112AC08091F3
:1029400084038F702FEF280F263008F0D8C08093B3
:10295000E9002091EB0020FF1CC0933021F480910E
:10296000EB00806214C09091EB0090619093EB00BB
:1029700021E030E0A90102C0440F551F8A95E2F71B
:102980004093EA001092EA008091EB008860809307
:10299000EB001092E9008091E800877F8093E800C7
:1029A0000E94D912ACC08111AAC0109182031F7776
:1029B0008091E3008078812B8093E3008091E80090
:1029C000877F8093E8000E94D9128091E80080FF01
:1029D000FCCF8091E30080688093E300111102C076
:1029E00082E001C083E080937F0389C080588230F9
:1029F00008F085C080918203909183038C3D53E061
:102A0000950779F583E08A838AE289834FB7F89442
:102A1000DE01139620E03EE051E2E32FF0E0509318
:102A20005700E49120FF03C0E295EF703F5FEF7025
:102A30008E2F90E0EA3010F0C79601C0C0968D93BB
:102A40009D932F5F243149F74FBF8091E800877F26
:102A50008093E8006AE270E0CE0101960E9478134C
:102A600016C06091840370918503AE014F5F5F4F84
:102A70000E943812BC01892B09F441C09091E800F2
:102A8000977F9093E80089819A810E94D613809164
:102A9000E8008B778093E80032C0803881F5809120
:102AA000E800877F8093E80080917B038093F100AA
:102AB0008091E8008E7772CF811121C080918203CE
:102AC0009091830399270297D4F48091E800877F3F
:102AD0008093E8008091820380937B030E94D91247
:102AE00080917B03811106C08091E30087FD02C0C5
:102AF00081E001C084E080937F030E948B1080916D
:102B0000E80083FF0AC08091E800877F8093E80097
:102B10008091EB0080628093EB00AA960FB6F89448
:102B2000DEBF0FBECDBFDF91CF911F9108950E94F0
:102B300005160E940D16E0EEF0E080818160808332
:102B4000E8EDF0E080818F77808319BCA7EDB0E0DD
:102B50008C918E7F8C9380818F7E808310927E03F8
:102B600008950F931F93CF93DF930E9405160E9441
:102B70000D16C8EDD0E088818F77888388818068C2
:102B8000888388818F7D888319BC10927F0310927F
:102B90007B0310927D0310927C0300EE10E0F8019D
:102BA00080818B7F808388818160888342E060E0C0
:102BB00080E00E94A412E1EEF0E080818E7F8083AD
:102BC000E2EEF0E080818160808380818860808394
:102BD000F80180818E7F8083888180618883DF9186
:102BE000CF911F910F910895E8EDF0E080818F7EE5
:102BF0008083E7EDF0E080818160808384E082BFA4
:102C000081E080937E030C94B115E8EDF0E08081C3
:102C10008E7F80831092E20008951092DA00109265
:102C2000E10008951F920F920FB60F9211242F9377
:102C30003F934F935F936F937F938F939F93AF9344
:102C4000BF93EF93FF938091E10082FF0BC08091CF
:102C5000E20082FF07C08091E1008B7F8093E1005A
:102C60000E94DF168091DA0080FF1FC08091D8009B
:102C700080FF1BC08091DA008E7F8093DA00809104
:102C8000D90080FF0DC080E189BD82E189BD09B412
:102C900000FEFDCF81E080937F030E947E1005C07F
:102CA00019BC10927F030E9487108091E10080FF81
:102CB00019C08091E20080FF15C08091E2008E7FF4
:102CC0008093E2008091E20080618093E200809135
:102CD000D80080628093D80019BC85E080937F0380
:102CE0000E945B118091E10084FF30C08091E2007E
:102CF00084FF2CC080E189BD82E189BD09B400FE5A
:102D0000FDCF8091D8008F7D8093D8008091E10025
:102D10008F7E8093E1008091E2008F7E8093E200BD
:102D20008091E20081608093E20080917B038823A0
:102D300011F084E007C08091E30087FD02C081E0CC
:102D400001C083E080937F030E9470118091E100B5
:102D500083FF24C08091E20083FF20C08091E100C6
:102D6000877F8093E10082E080937F0310927B0352
:102D70008091E1008E7F8093E1008091E2008E7F60
:102D80008093E2008091E20080618093E20042E063
:102D900060E080E00E94A4120E948A10FF91EF91EF
:102DA000BF91AF919F918F917F916F915F914F9163
:102DB0003F912F910F900FBE0F901F90189508957F
:102DC000CF9380917F038823A1F0C091E900CF7059
:102DD0009091EC00892F817090FD80E8C82B1092B3
:102DE000E9008091E80083FD0E943714CF70C09302
:102DF000E900CF9108959093800280937F02089517
:102E0000E0917F02F0918002309721F00190F081F3
:102E1000E02D099480E00895EF92FF920F931F93A5
:102E2000CF93DF93E0917F02F09180023097B1F170
:102E30008C010280F381E02D09958091750382FF5A
:102E40002DC080FF04C080E497E00E94BF05E80128
:102E500010E28AE3E82E87E0F82E8091750380FF68
:102E60000BC088811F928F93FF92EF920E945806A9
:102E70000F900F900F900F90115021961111EDCFE0
:102E80008091750380FF0AC088E397E0DF91CF91BE
:102E90001F910F91FF90EF900C94BF05DF91CF91A0
:102EA0001F910F91FF90EF900895CF93DF932091A2
:102EB0007D0230917E022817390709F190937E0236
:102EC00080937D02E0917F02F09180023097B9F00B
:102ED000EC010680F781E02D09958091750382FF52
:102EE0000EC080FF0CC0DF93CF938AE297E09F93E0
:102EF0008F930E9458060F900F900F900F90DF91C4
:102F0000CF910895CF93DF9320917B0230917C0283
:102F10002817390709F190937C0280937B02E09196
:102F20007F02F09180023097B9F0EC010084F185C6
:102F3000E02D09958091750382FF0EC080FF0CC0C3
:102F4000DF93CF938AE197E09F938F930E94580677
:102F50000F900F900F900F90DF91CF9108950C94E8
:102F600058180E94E6230C94E20ABF92CF92DF9297
:102F7000EF92FF920F931F93CF93DF9300D000D077
:102F80001F92CDB7DEB70E940C0B02E812E0F12CC5
:102F90008F2D0E94EF0AB82EF801C080C82639F4A0
:102FA000F3940F5F1F4FF0E1FF12F2CF30C080911A
:102FB000750381FD0E945918D12CEE24E3948C2DC9
:102FC0008E21F9F0D982FA8291E08B2D8E2109F4BD
:102FD00090E09B830E94EF238160782F9D838C83F8
:102FE00049815A816B818D810E948F1849815A8154
:102FF0006B817C818D810E948723F80180818E25E1
:103000008083D394EE0CF8E0DF12D9CFC9CF8FEFD5
:1030100089838A831B820E94EF238160782F9D839E
:103020008C8349815A816B818D810E948F180E9407
:1030300086230E94001790918102891741F10E9416
:103040000017809381029091750392FF0EC090FF4C
:103050000CC01F928F938BE497E09F938F930E94F5
:1030600058060F900F900F900F90809181020F9053
:103070000F900F900F900F90DF91CF911F910F91B4
:10308000FF90EF90DF90CF90BF900C9498230F901B
:103090000F900F900F900F90DF91CF911F910F9194
:1030A000FF90EF90DF90CF90BF9008950C94FD0AB1
:1030B0000895EF92FF920F931F93CF93DF9384E6CF
:1030C00097E00E94BF05C0E0D0E08CE2E82E81E0EE
:1030D000F82E06E517E08C2F0E94EF0A0E94742359
:1030E000FF92EF921F928F93DF93CF931F930F93D3
:1030F0000E94580621968DB79EB708960FB6F89491
:103100009EBF0FBE8DBFC031D10529F7DF91CF9192
:103110001F910F91FF90EF90089508950895CF9318
:10312000DF93CDB7DEB72B970FB6F894DEBF0FBE97
:10313000CDBF942F4F83252F588769877A878B8738
:103140004A855B85452B31F02F3F31F481E09F3F6D
:1031500019F403C081E001C080E080FD07C04F8109
:10316000588569857A858B850E948723DE011196B3
:1031700086E0FD0111928A95E9F785E0FE01379618
:1031800001900D928A95E1F749815A816B817C818A
:103190008D819E810E94821F2B960FB6F894DEBF10
:1031A0000FBECDBFDF91CF910895CF93882309F44F
:1031B00065C0C82F8CEF8C0F813A20F080E58C0F12
:1031C0008E3248F48C2F0E94C025811157C08C2F5D
:1031D0000E946A220CC080E28C0F883058F4C770BD
:1031E00081E001C0880FCA95EAF70E940F23CF91B2
:1031F0000C9449238BE58C0F833078F4C53A29F081
:10320000C63A31F083E890E005C081E890E002C062
:1032100082E890E0CF910C94551788E58C0F8731A8
:1032200068F5C83A89F0C93A91F0CA3A99F0CB3AB0
:10323000A1F0CC3AA9F0CD3AB1F0CE3AB9F0CF3AFC
:10324000C1F080E090E017C082EE90E014C089EEFB
:1032500090E011C08AEE90E00EC085EB90E00BC0CC
:1032600086EB90E008C083EB90E005C084EB90E033
:1032700002C087EB90E0CF910C948217CF91089514
:10328000882349F19CEF980F913A20F090E5980F30
:103290009E3218F40E94BA220DC090E2980F983026
:1032A00058F4877091E001C0990F8A95EAF7892F49
:1032B0000E9415230C9449239BE5980F933020F42A
:1032C00080E090E00C945517885A873120F480E014
:1032D00090E00C9482170895882321F00E940F2318
:1032E0000C9449230895882321F00E9415230C94FF
:1032F000492308950E942F230E94FE220E94492301
:1033000080E090E00E94551780E090E00C948217D6
:103310000E941F230C947A19CF92DF92EF92FF92B2
:103320000F931F93CF93DF9300D000D01F92CDB7A0
:10333000DEB76C010E949A238111EAC285E0F60192
:10334000DE01119601900D928A95E1F7F601408118
:103350005181238134812115310531F05F3F31F4F2
:1033600081E04F3F19F403C081E001C080E080FD9F
:10337000CFC2F601F280E580E2948FE0E822498333
:103380005A83FB82722F3D832C836F2D8D810E9487
:10339000E6218C010E94E5210E94D520E12FE295D3
:1033A000EF708E2F90E0FC01E75BFE4F0C9413262C
:1033B000812F807F1F70882311F01295107FFF20CE
:1033C00049F0112309F43BC2812F0E9422230E945D
:1033D000492335C2802F0E944019112309F498C255
:1033E000812F0E9428230F900F900F900F900F9025
:1033F000DF91CF911F910F91FF90EF90DF90CF90D1
:103400000C944923812F807F1F70803211F0129518
:10341000107F002319F0013009F12BC0FF20A9F023
:10342000EE2059F1F1E0812FEF1228C00F900F909C
:103430000F900F900F90DF91CF911F910F91FF9000
:10344000EF90DF90CF900C943223EE2021F021E01A
:10345000E21609F45DC20E9435232DC0FF20E9F079
:1034600085E08E1508F454C20E940C23812329F0B4
:1034700022C0FF20F1F0E11015C0812F0F900F90B6
:103480000F900F900F90DF91CF911F910F91FF90B0
:10349000EF90DF90CF900C946C1994E09E1508F497
:1034A00037C209C0F601858180FFC9C18F7085834D
:1034B000E4CFE110D7C1812F4AC1812F869586952F
:1034C000837019F08130B9F023C2FF2019F0C801D0
:1034D000937002C080E090E00F900F900F900F90DB
:1034E0000F90DF91CF911F910F91FF90EF90DF90A0
:1034F000CF900C945517FF2019F0C801937002C0AB
:1035000080E090E00F900F900F900F900F90DF9160
:10351000CF911F910F91FF90EF90DF90CF900C947F
:103520008217812F837009F070C0F110F1C1202F34
:10353000229526952770220F220F602F6F70862FFD
:1035400090E0A0E0B0E06C017D01022E04C0CC0C44
:10355000DD1CEE1CFF1C0A94D2F704FF12C08FE0A2
:1035600090E0A0E0B0E004C0880F991FAA1FBB1F25
:103570002A95D2F7BC01CD01609570958095909504
:1035800003C060E070E0CB01169516951370123001
:10359000B1F040F56C297D298E299F29113031F138
:1035A0000F900F900F900F900F90DF91CF911F9180
:1035B0000F91FF90EF90DF90CF900C94FA206C2940
:1035C0007D298E299F290F900F900F900F900F90BB
:1035D000DF91CF911F910F91FF90EF90DF90CF90EF
:1035E0000C9414210E94FA20C701B6010F900F908D
:1035F0000F900F900F90DF91CF911F910F91FF903F
:10360000EF90DF90CF900C94E020FF2019F0812FF5
:10361000817001C08695882309F47AC1202F2295F4
:1036200026952770220F220F602F6F70862F90E053
:10363000A0E0B0E06C017D01022E04C0CC0CDD1CCA
:10364000EE1CFF1C0A94D2F704FF12C08FE090E03A
:10365000A0E0B0E004C0880F991FAA1FBB1F2A95E5
:10366000D2F7BC01CD01609570958095909503C00F
:1036700060E070E0CB011695169513701230B1F032
:1036800040F56C297D298E299F29113031F10F9049
:103690000F900F900F900F90DF91CF911F910F918E
:1036A000FF90EF90DF90CF900C94C1216C297D2981
:1036B0008E299F290F900F900F900F900F90DF9100
:1036C000CF911F910F91FF90EF90DF90CF900C94CE
:1036D000D3210E94C121C701B6010F900F900F9016
:1036E0000F900F90DF91CF911F910F91FF90EF906E
:1036F000DF90CF900C94AF21003FC1F128F480E41B
:10370000800F803250F096C0023F09F45EC008F48A
:1037100049C0033F09F46CC08DC0F02FF071EF2E4B
:10372000812F8F71FF2051F00E944821802FEE20C1
:1037300019F08295807FA2CE8F70A0CE0E94692161
:10374000802FEE2019F08295807F01C08F700F903E
:103750000F900F900F900F90DF91CF911F910F91CD
:10376000FF90EF90DF90CF900C947319FF20A9F099
:1037700024E02E1508F4CCC0812F8F710F900F908C
:103780000F900F900F90DF91CF911F910F91FF90AD
:10379000EF90DF90CF900C948E2185E08E1508F489
:1037A000B7C0EACFFF2099F0812F8F710F900F9053
:1037B0000F900F900F90DF91CF911F910F91FF907D
:1037C000EF90DF90CF900C944821FF2069F3812F78
:1037D0008F710F900F900F900F900F90DF91CF91FE
:1037E0001F910F91FF90EF90DF90CF900C94692183
:1037F000FF2089F0812F8F710F900F900F900F9005
:103800000F90DF91CF911F910F91FF90EF90DF907C
:10381000CF900C9433210F900F900F900F900F903A
:10382000DF91CF911F910F91FF90EF90DF90CF909C
:103830000C942E21FF2099F0EE2009F4B5CF802FB3
:103840000F900F900F900F900F90DF91CF911F91DD
:103850000F91FF90EF90DF90CF900C94D518EE2051
:1038600009F4B5CF802F0F900F900F900F900F900D
:10387000DF91CF911F910F91FF90EF90DF90CF904C
:103880000C944019412F4F70602FC6010E945B2499
:103890000F900F900F900F900F90DF91CF911F918D
:1038A0000F91FF90EF90DF90CF900C94302001119A
:1038B0002FC0FF2069F10E9488199FEFE0E7F2E036
:1038C0009150E040F040E1F700C000000F900F90F1
:1038D0000F900F900F90DF91CF911F910F91FF905C
:1038E000EF90DF90CF900C943C24412F4F70602FCD
:1038F000C6010F900F900F900F900F90DF91CF9116
:103900001F910F91FF90EF90DF90CF900C945E2469
:103910000F900F900F900F900F90DF91CF911F910C
:103920000F91FF90EF90DF90CF9008951F93CF936A
:10393000DF9300D000D01F92CDB7DEB7942F49831C
:10394000252F5A836B837C838D834C815D81452B2E
:1039500031F02F3F31F481E09F3F19F403C081E043
:1039600001C080E0182F117080FD31C049815A815B
:103970006B817C818D810E94E621292F22952F70F9
:103980002C3030F42A30A0F42250223030F022C003
:103990002C30C9F02F30B9F01DC0853A28F484309E
:1039A000C0F4823028F415C090E2980F983088F067
:1039B000883E30F4803E68F48450813A58F409C05F
:1039C000803F41F406C093FB112710F903C010E0BB
:1039D00001C011E0812F0F900F900F900F900F906A
:1039E000DF91CF911F910895CF93DF9300D000D046
:1039F0001F92CDB7DEB70F900F900F900F900F90E2
:103A0000DF91CF910895CF93DF9300D000D000D005
:103A1000CDB7DEB726960FB6F894DEBF0FBECDBF8A
:103A2000DF91CF9108951F93CF93DF93C0919202BE
:103A300016E080919302C81799F0D0E01C9FF00126
:103A40001D9FF00D1124EC56FD4F40815181628184
:103A50007381848195810E94031D2196C770E9CFEF
:103A6000DF91CF911F9108954091C4025091C502FA
:103A70006091C6027091C7028091C8029091C902FC
:103A80000C94031D0F931F93CF93DF938091C90272
:103A900082958F7009F05DC08091C602882309F479
:103AA00058C080919202109193026091C40270916B
:103AB000C502C091C702D091C80291E06F3F09F0E2
:103AC00090E0292F06E0811709F443C0209721F0E8
:103AD0007F3F21F030E003C031E001C0322F90E0A1
:103AE00030FD34C0089FF001099FF00D1124DF0163
:103AF000AC56BD4F11963C911197371327C03C919E
:103B0000361324C012963C91129731111FC01396A0
:103B10004D915C9114974C1B5D0B483C5105B0F4E2
:103B20008091C9028F7080618093C902E756FD4F72
:103B300080818F708061808384EC92E00E948C1978
:103B4000DF91CF911F910F910C94131D01968770F7
:103B5000BACFDF91CF911F910F9108959F92AF92AD
:103B6000BF92CF92DF92EF92FF920F931F93CF936A
:103B7000DF93CDB7DEB761970FB6F894DEBF0FBE07
:103B8000CDBF8C0185E0F801DE011D9601900D92FC
:103B90008A95E1F7F80140815181F280C380D48099
:103BA0009091C4026091C5022091C7023091C80271
:103BB0002115310531F06F3F31F481E09F3F19F459
:103BC00003C081E001C080E0F82FF1709F2E80FDDE
:103BD00052C184ECA82E82E0B82EE090C602F60115
:103BE000E21BF30BEE2009F4E8C08091C902E83C27
:103BF000F10508F0A4C0282F207F09F053C0561308
:103C000013C0491311C0EF2CF1100EC08F708061EA
:103C10008093C9020E94341DC5010E948C198091B5
:103C2000C902F80185835BC1C114D10431F05F3F43
:103C300031F481E04F3F19F403C081E001C080E01E
:103C400080FD03C081E08F2502C080E090E0F82F66
:103C5000F170EF2E80FF1CC08091920220919302A0
:103C600036E0821709F418C190E0389FF001399FBF
:103C7000F00D1124EC56FD4F6181561306C0608192
:103C8000461303C06281F61203C001968770E9CF24
:103C9000EF2CFF2009F423C18091C9028160809339
:103CA000C90262C0561306C0491304C0F11002C015
:103CB000F801A7C04D875E87FF867C2DD98AC88A08
:103CC0006F2D89890E94961C882399F1FF2089F124
:103CD0002091C902822F82958F7090E0029774F034
:103CE0008091C4029091C50298878F831986DB86E4
:103CF000CA862C87CE0107960E948C1986E0F801AF
:103D0000A4ECB2E001900D928A95E1F70E94421D69
:103D10000E94341D11C0561749F14D875E87FF86FA
:103D20007C2DD98AC88A6F2D89890E94961C8111A1
:103D30002CC0C8010E948C19EE24E394D0C0282F17
:103D4000207F49F77C2DD98AC88A6F2D89890E94E6
:103D5000F41C84EC92E00E948C1986E0F50111922B
:103D60008A95E9F70E94341DE12CB9C04913D5CFDB
:103D7000F110D3CFF8018583C8010E948C1986E029
:103D8000F50111928A95E9F7AAC0FF2091F22091DE
:103D9000C902822F82958F7090E002970CF4AECF0B
:103DA0008091C4029091C5029A8389831B82DD822F
:103DB000CC822E83CE0101969FCFE83CF10508F01E
:103DC0004BC0EF2CFF2009F4B4CF561330C0491379
:103DD0002EC02091C90220FD21C0822F82958F70B4
:103DE000482F50E041155105C9F0F80125834F30A7
:103DF000510541F08F5F982F9295907F822F8F70A1
:103E0000892B8583C8010E948C1986E0F801A4ECF7
:103E1000B2E001900D928A95E1F72AC086E0F801A0
:103E2000A4ECB2E001900D928A95E1F758C04D875D
:103E30005E87FF867C2DD98AC88A6F2D89890E946A
:103E4000961C81115BCF8091C90281608093C90269
:103E5000C8010E948C1943C07C2DD98AC88A6F2D55
:103E600089890E94F41C86E0F50111928A95E9F790
:103E70000E94341D34C0FF2009F45BCF4D875E875C
:103E8000FF867C2DD98AC88A6F2D89890E94961C4D
:103E9000882309F44ECF32CF7C2DD98AC88A6F2D62
:103EA00089890E94E621292F22952F70223028F43B
:103EB0009F7039F0811105C00BC0243028F49F7029
:103EC00049F4805E883020F0C8010E948C199E2C35
:103ED000E92C05C0F8019581907F99F7F9CF8E2DD7
:103EE00061960FB6F894DEBF0FBECDBFDF91CF91C4
:103EF0001F910F91FF90EF90DF90CF90BF90AF9008
:103F00009F9008951F93CF93DF93CDB7DEB72C9783
:103F10000FB6F894DEBF0FBECDBF4F8358876987B9
:103F20007A878B879C87CE0107960E94AE1D8823D7
:103F3000D1F09F8188852A853B85232B31F08F3FE7
:103F400031F481E09F3F19F403C081E001C080E0BB
:103F500080FD47C04F81588569857A858B859C8512
:103F60000E94031D3EC086E0FE013796DE011196D9
:103F700001900D928A95E1F7FF81E8856A857B853E
:103F80006115710531F0EF3F31F481E0FF3F19F425
:103F900003C081E001C080E080FD23C02091930236
:103FA00030E0C9010196877099274091920250E054
:103FB00084179507F1F1F983EA837D836C8396E09A
:103FC000929FD001939FB00D1124AC56BD4FFE01BE
:103FD000319601900D929A95E1F7809393020E9499
:103FE000131D16E08091920290919302891771F14E
:103FF000189FC00111248C569D4F0E94AE1D88232E
:1040000029F1E09192021E9FF0011124EC56FD4F20
:104010004081518162817381848195810E94031D59
:104020008091920290E00196877099278093920286
:10403000D9CF0E9488191092930210929202E4EC58
:10404000F2E086E0DF011D928A95E9F72C960FB623
:10405000F894DEBF0FBECDBFDF91CF911F910895C1
:10406000DF92EF92FF920F931F93CF93DF93FC01A8
:10407000892B09F488C0E12CF12CDD24D394EF01C5
:1040800021968491853709F460C058F4843708F08C
:104090004EC0843008F068C08130D1F0823071F1B8
:1040A00072C0883709F45BC050F4863709F453C0F6
:1040B000873709F068C08E2D0E941C2352C09CE7F0
:1040C000980F903708F05FC08F770E9440194EC05C
:1040D0008F010E5F1F4FFE01849190E2980F983080
:1040E00050F48770FD2D01C0FF0F8A95EAF78F2FDE
:1040F0000E94222315C00E94D51814C08F010E5FA4
:104100001F4FFE01849190E2980F983068F48770F9
:10411000FD2D01C0FF0F8A95EAF78F2F0E942823FB
:104120000E944923E80122C00E944019FBCFCF0121
:104130000296FE01C491CC2361F0EFE9FFE03197D4
:10414000F1F700C00000C150F6CFCF010296FE018A
:10415000F490EC010BC00E940C23E82E07C00E94D3
:104160001F230E94492302C00E94D5188F2D882347
:1041700041F0EFE9FFE03197F1F700C00000815016
:10418000F6CFFE017CCFDF91CF911F910F91FF9071
:10419000EF90DF90089560934A0370934B038093F0
:1041A0004C0390934D030C949723089560934E0312
:1041B00070934F0380935003909351030C94962374
:1041C0000F931F9300914E0310914F0320915003C2
:1041D00030915103602B712B822B932B60934E03F4
:1041E00070934F0380935003909351031F910F914D
:1041F0000C9496230F931F9300914E0310914F033D
:104200002091500330915103602371238223932323
:1042100060934E0370934F03809350039093510328
:104220001F910F910C9496230F931F9300914E03AF
:1042300010914F0320915003309151036027712753
:104240008227932760934E0370934F03809350030C
:10425000909351031F910F910C94962360E070E0AE
:10426000CB010C94CB200F931F9341E050E060E012
:1042700070E08A019B0104C0000F111F221F331F31
:104280008A95D2F7C901B8011F910F910C94CB20E8
:104290000F931F9341E050E060E070E004C0440FD2
:1042A000551F661F771F8A95D2F780914A03909118
:1042B0004B03A0914C03B0914D038A019B01082B45
:1042C000192B2A2B3B2BC901B8011F910F910C947C
:1042D000CB200F931F9341E050E060E070E004C0FA
:1042E000440F551F661F771F8A95D2F7409550954A
:1042F0006095709580914A0390914B03A0914C0377
:10430000B0914D038A019B01082319232A233B23E3
:10431000C901B8011F910F910C94CB200F931F93EB
:1043200041E050E060E070E004C0440F551F661F9C
:10433000771F8A95D2F780914A0390914B03A09101
:104340004C03B0914D038A019B01082719272A27A6
:104350003B27C901B8011F910F910C94CB200F93FB
:104360001F9300914A0310914B0320914C0330910D
:104370004D03602B712B822B932B1F910F910C946B
:10438000CB200F931F9300914A0310914B03209170
:104390004C0330914D0360237123822393231F919B
:1043A0000F910C94CB200F931F9300914A0310910F
:1043B0004B0320914C0330914D03602771278227D6
:1043C00093271F910F910C94CB2008958F929F9269
:1043D000AF92BF92DF92EF92FF920F931F93CF9312
:1043E000DF9300D000D01F92CDB7DEB76B837C8304
:1043F0008D838A018C819D81892B31F01F3F31F49F
:1044000081E04F3F19F403C081E001C080E080FFEC
:1044100003C080E090E04DC08B818823D1F1809073
:104420004A0390904B03A0904C03B0904D038091B1
:104430004E0390914F03A0915003B0915103882AED
:10444000992AAA2ABB2A8FE1E82EF12CD501C401B2
:104450000E2C04C0B695A795979587950A94D2F728
:1044600080FD06C081E0E81AF10880F7D12C07C072
:10447000DE2CB8018E2D0E946106019799F388E029
:10448000189FF0011124E653FD4FE00FF11DD0827B
:1044900009C088E0189FF0011124E653FD4FE00F9A
:1044A000F11DD08009831A8369817A818D2D0E9444
:1044B00061060F900F900F900F900F90DF91CF91AA
:1044C0001F910F91FF90EF90DF90BF90AF909F9062
:1044D0008F90089590911401992379F1909115018D
:1044E000992359F1982F9695969596959F31A1F01D
:1044F000E0911601F0911701E90FF11D877021E09D
:1045000030E0A90102C0440F551F8A95E2F7CA01A5
:104510009181892B818308959091750390FF29C023
:104520001F928F9380E997E09F938F930E94580684
:104530000F900F900F900F900895209116013091D9
:104540001701F90132969FEF40E05191851789F0EC
:104550009F3F19F4511101C0942F4F5F4E31A9F7BD
:104560009F3F39F0F901E90FF11D97FDFA9582831C
:104570000895089590911401992381F19091150166
:10458000992361F1982F9695969596959F31A9F06C
:10459000E0911601F0911701E90FF11D877021E0FC
:1045A00030E0A90102C0440F551F8A95E2F7CA0105
:1045B000809591818923818308959091750390FF5F
:1045C0001CC01F928F9382E797E09F938F930E9466
:1045D00058060F900F900F900F900895E0911601DC
:1045E000F09117019F01225E3F4F9281891301C014
:1045F00012823196E217F307C1F7089581E090E047
:10460000E0911601F0911701E80FF91F1082019651
:1046100080329105A9F708958091740308959091CF
:104620007403892B8093740308958095909174038B
:1046300089238093740308958093740308951092DE
:104640007403089590917303892B809373030895E5
:10465000809590917303892380937303089510923A
:10466000730308958093520308951092520308959E
:104670008091160190911701FC0131969C01205EFA
:104680003F4F80E0919191118F5FE217F307D1F7CF
:104690000895E0911601F0911701809174038083D1
:1046A000E0911601F0911701908180917303892B9D
:1046B000808380915203882361F0E0911601F0918C
:1046C00017019081892B80830E94382381111092D9
:1046D000520380911601909117010C940C1790933E
:1046E00035018093340108958295982F937344E0A7
:1046F000949F900111248C7C86958695282B822F7F
:104700008575880F2A7A2695822B08950895CF9370
:10471000DF9300D000D01F92CDB7DEB70F900F907F
:104720000F900F900F90DF91CF9108950895089505
:104730000C94561880E0089583B7817F8C6083BF06
:1047400083B7816083BF7894889583B78E7F83BF5A
:104750000895CF930E948D180E940C0B0E948E1812
:10476000C0E08C2F0E94EF0A811104C0CF5FC031DE
:10477000C1F701C081E0CF9108950E94F50A0C9421
:1047800088191F920F920FB60F9211248F939F9347
:10479000AF93BF938091760390917703A0917803B4
:1047A000B09179034196A11DB11D8093760390933A
:1047B0007703A0937803B0937903BF91AF919F9152
:1047C0008F910F900FBE0F901F90189582E084BDBF
:1047D00093E095BD9AEF97BD80936E0008952FB733
:1047E000F8948091760390917703A0917803B0912B
:1047F00079032FBF08952FB7F894609176037091D5
:10480000770380917803909179032FBF08959C01DD
:104810004FB7F8948091760390917703A091780335
:10482000B09179034FBF821B930B089578941F9228
:104830000F920FB60F9211248F939F93AF93BF9354
:104840008091760390917703A0917803B0917903DA
:104850000196A11DB11D8093760390937703A093D9
:104860007803B0937903BF91AF919F918F910F908F
:104870000FBE0F901F9018950E949715F89487E728
:1048800097E7909301088093000887E090EBDC01A4
:104890008093880390938903A0938A03B0938B033A
:1048A0009CE088E10FB6F894A895809360000FBE55
:1048B00090936000FFCF80E090E008950895CF933B
:1048C000C82F1F928F9384EB97E09F938F930E9442
:1048D000580681E090E0A0E0B0E0BC01CD0104C04A
:1048E000660F771F881F991FCA95D2F70E94D6209E
:1048F0000F900F900F900F90CF910C948819CF9339
:104900008732A8F58E3108F02BC1803109F49FC0A1
:10491000F8F4873009F464C0A8F4863009F024C1A3
:1049200080917503817F8E7F8093750389EB97E07B
:104930000E94BF058BE99AE00E94BF0581E0809349
:104940007A034CC08B30F1F18E3009F46CC00CC18D
:10495000863109F4B0C020F4813109F4EDC004C1FE
:10496000893109F491C08B3109F449C0FDC0883305
:1049700049F150F4893209F4F1C0853309F4EEC0ED
:10498000873209F0F1C0EAC0833409F4E7C028F4A3
:104990008A3308F4E9C08953E4C0883409F0E4C0DC
:1049A0000E9488198AE89AE00E94BF052FEF83EDE4
:1049B00090E3215080409040E1F700C000000E9449
:1049C0003C240CC084ED97E05CC081E79AE00E9433
:1049D000BF0580917503816080937503C1E0C9C0F4
:1049E00080917503C82FC17080FFEFCF8DE79AE0EB
:1049F0000E94BF0580917503817F8E7F3DC090919D
:104A0000750391FBCC27C0F981E0C827892FC0FB33
:104A100081F980937503CC2319F084E69AE027C0CE
:104A200086E59AE02EC09091750392FBCC27C0F9E1
:104A300081E0C827892FC0FB82F980937503CC23BE
:104A400019F087E49AE013C087E39AE01AC09091C6
:104A5000750393FBCC27C0F981E0C827892FC0FBE1
:104A600083F980937503CC2351F08BE29AE00E9486
:104A7000BF05809175038160809375037AC08EE1D4
:104A80009AE00E94BF05AACF8FE09AE00E94BF057E
:104A900089EE99E00E94BF0581EA99E00E94BF0576
:104AA00089E799E00E94BF058DE299E00E94BF0569
:104AB00082E099E0E6CF84EF98E00E94BF050E9473
:104AC00000171F928F938AED98E09F938F930E9417
:104AD0005806809114011F928F9383EC98E09F9366
:104AE0008F930E94580680917A021F928F9380EBD9
:104AF00098E09F938F930E945806809115011F9212
:104B00008F938DE998E09F938F930E9458060E949F
:104B1000FB239F938F937F936F9386E898E09F93F7
:104B20008F930E9458068DB79EB746960FB6F8949D
:104B30009EBF0FBE8DBF52CF0E948819C091150134
:104B400081E0C827C0931501CC2329F08CE798E0B9
:104B50000E94BF050EC081E798E093CF80E001C0BE
:104B60008D510E945F243ACF8FE698E00E94BF05E6
:104B7000C0E08C2FCF91089580E008950C94BC255F
:104B8000CF93C82F80917A03882319F0813059F090
:104B900042C0E0911601F09117018081823261F0EC
:104BA0008434D9F509C0E0911601F0911701808194
:104BB000823211F0843461F48C2F0E94BE25811161
:104BC00004C08C2F0E947F2424C081E090E021C08B
:104BD0008C2F0E94BC2581111BC0C43189F018F4B0
:104BE000CB3029F010C0C93259F0C83361F489EBD9
:104BF00097E00E94BF0580EB97E00E94BF0508C0C8
:104C000010927A030CC08EEA97E00E94BF0507C09D
:104C100081E0817006C010927A0380E002C080E0DB
:104C2000F8CFCF910895EE0FFF1F0590F491E02D7E
:064C30000994F894FFCF87
:104C36000080FFFF0559010000FFB70E240FBA0ED2
:104C4600EF0EBB0E0101530340362239DA06A406E5
:104C560082064906D505EE05070627060000080068
:044C66000400020044
:106800008800EA44E944E244040005000600070069
:10681000080009000A000B000C000D000E000F001C
:1068200010001100120013001400150016001700CC
:10683000180019001A001B001C001D001E001F007C
:10684000200021002200230024002500260027002C
:10685000280029002A002B002C002D002E002F00DC
:10686000300031003200330034003500360037008C
:10687000380039003A003B003C003D003E003F003C
:1068800040004100420043004400450046004700EC
:10689000480049004A004B004C004D004E004F009C
:1068A000500051005200530054005500560057004C
:1068B000580059005A005B005C005D005E005F00FC
:1068C0006000610062006300640065A185006700EC
:1068D000680069006A006B006C006D006E006F005C
:1068E0007000710072007300890087008A008B00BD
:1068F000E000E100E200E300E400E500E600E7007C
:106900000100010001000100EA4401000100E2442D
:106910000100010001000100460001004A004B0097
:10692000010001004700480001000100E9440100A6
:106930000100010001000100010001003A003B00DC
:106940003C003D003E003F0040004100420043004B
:10695000010035004C0039000100440045005200A0
:1069600049000100010050004F0029004D004E0079
:1069700051000100010001000100010001000100BF
:1069800001000100010001000100010001000100FF
:1069900001000100010001000100010001004D00A3
:1069A0004A004E004B0001000100010001000100FF
:1069B00001000100010001000100010001000100CF
:1069C00001000100010001000100010001000100BF
:1069D00001000100010001000100010001000100AF
:1069E0000100010001000100490001000100010057
:1069F000010001000100010001000100010001008F
:00000001FF
